:020000040000FA
:020000001028C6
:020008000900ED
:100020008501831600308100E0308500FF308600B6
:10003000831207309F0010308500A2010030332862
:100040000B1182073A28B928D828C928D128DB28DB
:10005000E228EA28EF28F3285A2861280A291429D7
:10006000362989287E280B1D3328A000E630810020
:10007000200820280A30AD008B200A309620AD01E0
:1000800034302207840006088000220A0F39A200BB
:100090000508F039220485008009AD0A9620A208DF
:1000A000031D4028B1013430220784000608AB004C
:1000B0000A30332805122B080006031D73280B3065
:1000C00033280516220AB10AB10A0F39A200050821
:1000D000F039220410388500AD0A9620A208031DCD
:1000E0005328B1015328B001A900AA000F3E831C78
:1000F0007F280315F6202621103033280512F03012
:10010000290503195F280311F620B00E26210F30B0
:10011000332805125F280030A3000030A40003300C
:10012000A800E620A120AD0B8B280800FF30A3001B
:100130000030A4000330A800E620A120AD0B9628D3
:100140000800233084002808A000A003A0030008B2
:10015000840A0006840AA00BA928800023308400AA
:100160000B1DB028ED3081000B110930A7000130C4
:10017000332805120B1DBA28ED3081000B11A70B97
:10018000C228DD28800D031CC72802303328033025
:10019000332805160B1DCA28ED3081000B110430E1
:1001A000332805120B1DD228ED3081000B11BF281A
:1001B0000516053033280512BF28840A0930A70028
:1001C000063033280516A80BB02808000E30AE0004
:1001D000073033280512AE0BF128083033280516F6
:1001E0000800093033280516073033280319002981
:1001F000A90E2908AA00AB0E3108013EA30002296E
:100200003108A3000F30AA050330AE01B001B00AD7
:100210000C3033280516AA0C03181229B00DAE0AAB
:10022000AE0A0B290D303328051234302207840022
:100230002B080F393005031922292E08013EA4008E
:10024000031108002E08A4000315080003192B2928
:10025000300880042D2930098005A31723132308B3
:10026000B300F0302404B2000E30332805160130FC
:100270003206A400E6200330A800A1200130AD0022
:1002800096203308A3003208A400A415E62003300A
:06029000A800A1200800F7
:02400E00613F10
:00000001FF
